:020000040000FA
:100000000C9462000C948A000C948A000C948A0070
:100010000C948A000C948A000C948A000C948A0038
:100020000C948A000C948A000C948A000C948A0028
:100030000C948A000C948A000C948A000C948A0018
:100040000C94BE010C948A000C942E020C940802AD
:100050000C948A000C948A000C948A000C948A00F8
:100060000C948A000C948A000000000025002800EF
:100070002B0000000000240027002A0000000000E0
:1000800023002600290004040404040404040202DA
:100090000202020203030303030301020408102007
:1000A0004080010204081020010204081020000012
:1000B0000008000201000003040700000000000027
:1000C0000000B10311241FBECFEFD8E0DEBFCDBFCB
:1000D00011E0A0E0B1E0ECECF7E002C005900D9279
:1000E000A231B107D9F721E0A2E1B1E001C01D9230
:1000F000A83BB207E1F710E0C2E6D0E004C02197C8
:10010000FE010E94DE03C136D107C9F70E946002DA
:100110000C94E4030C9400003FB7F8948091B40170
:100120009091B501A091B601B091B70126B5A89BF9
:1001300005C02F3F19F00196A11DB11D3FBFBA2F79
:10014000A92F982F8827BC01CD01620F711D811D39
:10015000911D42E0660F771F881F991F4A95D1F7BE
:100160000895AF92BF92CF92DF92EF92FF920F93DA
:100170001F93CF93DF936C017B018B01040F151F3D
:10018000EB015E01AE18BF08C017D10759F06991A5
:10019000D601ED91FC910190F081E02DC601099509
:1001A000892B79F7C501DF91CF911F910F91FF90B6
:1001B000EF90DF90CF90BF90AF900895FC01538DEA
:1001C000448D252F30E0842F90E0821B930B541731
:1001D00010F0CF96089501970895FC01918D828DBE
:1001E000981761F0A28DAE0FBF2FB11D5D968C9157
:1001F000928D9F5F9F73928F90E008958FEF9FEF96
:100200000895FC01918D828D981731F0828DE80F51
:10021000F11D858D90E008958FEF9FEF0895FC010B
:10022000918D228D892F90E0805C9F4F821B9109D8
:100230008F739927089582E191E00E940F0121E0D8
:10024000892B09F420E0822F089580E090E0892B2B
:1002500029F00E941B0181110C9400000895FC01FB
:10026000A48DA80FB92FB11DA35ABF4F2C91848D17
:1002700090E001968F739927848FA689B7892C9374
:10028000A089B1898C91837080648C93938D848DC7
:10029000981306C00288F389E02D80818F7D8083CA
:1002A0000895EF92FF920F931F93CF93DF93EC018A
:1002B00081E0888F9B8D8C8D98131AC0E889F9890D
:1002C000808185FF15C09FB7F894EE89FF89608310
:1002D000E889F98980818370806480839FBF81E091
:1002E00090E0DF91CF911F910F91FF90EF900895D3
:1002F000F62E0B8D10E00F5F1F4F0F731127E02EAE
:100300008C8D8E110CC00FB607FCFACFE889F989E5
:10031000808185FFF5CFCE010E942F01F1CFEB8DBB
:10032000EC0FFD2FF11DE35AFF4FF0829FB7F894B9
:100330000B8FEA89FB8980818062CFCFCF93DF93D7
:10034000EC01888D8823B9F0AA89BB89E889F989ED
:100350008C9185FD03C0808186FD0DC00FB607FC22
:10036000F7CF8C9185FFF2CF808185FFEDCFCE0155
:100370000E942F01E9CFDF91CF9108951F920F9234
:100380000FB60F9211242F933F938F939F93AF93A8
:10039000BF938091B0019091B101A091B201B09151
:1003A000B3013091AF0123E0230F2D3758F50196AB
:1003B000A11DB11D2093AF018093B0019093B101B5
:1003C000A093B201B093B3018091B4019091B501B3
:1003D000A091B601B091B7010196A11DB11D809306
:1003E000B4019093B501A093B601B093B701BF914A
:1003F000AF919F918F913F912F910F900FBE0F90D2
:100400001F90189526E8230F0296A11DB11DD2CF8B
:100410001F920F920FB60F9211242F933F934F9379
:100420005F936F937F938F939F93AF93BF93EF935C
:10043000FF9382E191E00E942F01FF91EF91BF9124
:10044000AF919F918F917F916F915F914F913F916C
:100450002F910F900FBE0F901F9018951F920F9223
:100460000FB60F9211242F938F939F93EF93FF93C7
:10047000E0912201F09123018081E0912801F09127
:10048000290182FD1BC0908180912B018F5F8F73AA
:1004900020912C01821741F0E0912B01F0E0EE5EFB
:1004A000FE4F958F80932B01FF91EF919F918F913C
:1004B0002F910F900FBE0F901F9018958081F4CF51
:1004C000CF93DF93CDB7DEB7A1970FB6F894DEBF19
:1004D0000FBECDBF789484B5826084BD84B5816041
:1004E00084BD85B5826085BD85B5816085BD8091FF
:1004F0006E00816080936E00109281008091810077
:10050000826080938100809181008160809381006E
:10051000809180008160809380008091B100846030
:100520008093B1008091B00081608093B000809191
:100530007A00846080937A0080917A008260809350
:100540007A0080917A00816080937A0080917A00AD
:10055000806880937A001092C100E0912201F091AE
:10056000230182E08083E0911E01F0911F0110823F
:10057000E0912001F09121018FEC808310922A01FB
:10058000E0912601F091270186E08083E09124012B
:10059000F0912501808180618083E0912401F091B8
:1005A0002501808188608083E0912401F0912501FC
:1005B000808180688083E0912401F0912501808111
:1005C0008F7D80836CE9262E60E0362EF101249128
:1005D00078E8E72E70E0F72EF70184918823C9F0C0
:1005E00090E0880F991FFC01EE58FF4FA591B49140
:1005F000FC01E859FF4F459154913FB7F8949C9105
:10060000822F809598239C93FA019081892380837F
:100610003FBFE7EAF0E02491E3E9F0E0849188232A
:1006200099F090E0880F991FFC01EE58FF4FA591BB
:10063000B491FC01E859FF4F859194918FB7F894DC
:10064000EC91E22BEC938FBF8E01005E1F4F30E0E8
:10065000C32E30E0D32EE0EBF0E08491F1019491D1
:10066000F70124912223C9F0882359F0833009F43B
:1006700061C008F054C0813009F462C0823009F4CE
:1006800063C0E22FF0E0EE0FFF1FE458FF4FA5918B
:10069000B4918C91982381E009F480E019A2805DE7
:1006A00088A3F80101900020E9F73197AF01401BC2
:1006B000510BB80182E191E00E94B1000E948C00D0
:1006C0002B013C0184EF882E99249394A12CB12C0A
:1006D0000E948C006419750986099709683E734069
:1006E00081059105A8F3F1E08F1A9108A108B108DE
:1006F00028EE420E23E0521E611C711C81149104ED
:10070000A104B10429F7C114D10409F4A4CF0E94B3
:100710001B01882309F49FCF0E9400009CCF8730E3
:10072000B1F08830D1F0843009F0ABCF80918000F7
:100730008F7D03C0809180008F7780938000A1CF50
:1007400084B58F7784BD9DCF84B58F7DFBCF80919D
:10075000B0008F778093B00094CF8091B0008F7DF0
:10076000F9CFE2E1F1E01382128288EE93E0A0E09B
:10077000B0E084839583A683B78384E091E091837E
:10078000808385EC90E09587848784EC90E0978760
:10079000868780EC90E0918B808B81EC90E0938B4E
:1007A000828B82EC90E0958B848B86EC90E0978B2B
:1007B000868B118E128E138E148E0895EE0FFF1FEE
:1007C0000590F491E02D0994F894FFCF000000000B
:0E07D0005101B100DE009E010F01ED0001019C
:107E0000112484B714BE81FFF0D085E080938100F7
:107E100082E08093C00088E18093C10086E0809377
:107E2000C20080E18093C4008EE0C9D0259A86E02C
:107E300020E33CEF91E0309385002093840096BBD3
:107E4000B09BFECF1D9AA8958150A9F7CC24DD24C4
:107E500088248394B5E0AB2EA1E19A2EF3E0BF2EE7
:107E6000A2D0813461F49FD0082FAFD0023811F036
:107E7000013811F484E001C083E08DD089C08234E0
:107E800011F484E103C0853419F485E0A6D080C0E4
:107E9000853579F488D0E82EFF2485D0082F10E0AE
:107EA000102F00270E291F29000F111F8ED06801E7
:107EB0006FC0863521F484E090D080E0DECF843638
:107EC00009F040C070D06FD0082F6DD080E0C81688
:107ED00080E7D80618F4F601B7BEE895C0E0D1E017
:107EE00062D089930C17E1F7F0E0CF16F0E7DF06D8
:107EF00018F0F601B7BEE89568D007B600FCFDCFD4
:107F0000A601A0E0B1E02C9130E011968C91119780
:107F100090E0982F8827822B932B1296FA010C0160
:107F200087BEE89511244E5F5F4FF1E0A038BF0790
:107F300051F7F601A7BEE89507B600FCFDCF97BE46
:107F4000E89526C08437B1F42ED02DD0F82E2BD052
:107F50003CD0F601EF2C8F010F5F1F4F84911BD097
:107F6000EA94F801C1F70894C11CD11CFA94CF0C13
:107F7000D11C0EC0853739F428D08EE10CD085E9AC
:107F80000AD08FE07ACF813511F488E018D01DD067
:107F900080E101D065CF982F8091C00085FFFCCF94
:107FA0009093C60008958091C00087FFFCCF809118
:107FB000C00084FD01C0A8958091C6000895E0E648
:107FC000F0E098E1908380830895EDDF803219F02E
:107FD00088E0F5DFFFCF84E1DECF1F93182FE3DFCA
:107FE0001150E9F7F2DF1F91089580E0E8DFEE27F6
:047FF000FF270994CA
:027FFE00040479
:00000001FF
